Archive member included to satisfy reference by file (symbol)

c:/program files (x86)/atmel/studio/7.0/toolchain/avr8/avr8-gnu-toolchain/bin/../lib/gcc/avr/5.4.0/../../../../avr/lib/avrxmega6\libm.a(addsf3.o)
                              src/main.o (__subsf3)
c:/program files (x86)/atmel/studio/7.0/toolchain/avr8/avr8-gnu-toolchain/bin/../lib/gcc/avr/5.4.0/../../../../avr/lib/avrxmega6\libm.a(addsf3x.o)
                              c:/program files (x86)/atmel/studio/7.0/toolchain/avr8/avr8-gnu-toolchain/bin/../lib/gcc/avr/5.4.0/../../../../avr/lib/avrxmega6\libm.a(addsf3.o) (__addsf3x)
c:/program files (x86)/atmel/studio/7.0/toolchain/avr8/avr8-gnu-toolchain/bin/../lib/gcc/avr/5.4.0/../../../../avr/lib/avrxmega6\libm.a(divsf3.o)
                              src/main.o (__divsf3)
c:/program files (x86)/atmel/studio/7.0/toolchain/avr8/avr8-gnu-toolchain/bin/../lib/gcc/avr/5.4.0/../../../../avr/lib/avrxmega6\libm.a(divsf3x.o)
                              c:/program files (x86)/atmel/studio/7.0/toolchain/avr8/avr8-gnu-toolchain/bin/../lib/gcc/avr/5.4.0/../../../../avr/lib/avrxmega6\libm.a(divsf3.o) (__divsf3x)
c:/program files (x86)/atmel/studio/7.0/toolchain/avr8/avr8-gnu-toolchain/bin/../lib/gcc/avr/5.4.0/../../../../avr/lib/avrxmega6\libm.a(fixsfsi.o)
                              src/adc_sensors/adc_sensors.o (__fixsfsi)
c:/program files (x86)/atmel/studio/7.0/toolchain/avr8/avr8-gnu-toolchain/bin/../lib/gcc/avr/5.4.0/../../../../avr/lib/avrxmega6\libm.a(fixunssfsi.o)
                              c:/program files (x86)/atmel/studio/7.0/toolchain/avr8/avr8-gnu-toolchain/bin/../lib/gcc/avr/5.4.0/../../../../avr/lib/avrxmega6\libm.a(fixsfsi.o) (__fixunssfsi)
c:/program files (x86)/atmel/studio/7.0/toolchain/avr8/avr8-gnu-toolchain/bin/../lib/gcc/avr/5.4.0/../../../../avr/lib/avrxmega6\libm.a(floatsisf.o)
                              src/adc_sensors/adc_sensors.o (__floatunsisf)
c:/program files (x86)/atmel/studio/7.0/toolchain/avr8/avr8-gnu-toolchain/bin/../lib/gcc/avr/5.4.0/../../../../avr/lib/avrxmega6\libm.a(fp_inf.o)
                              c:/program files (x86)/atmel/studio/7.0/toolchain/avr8/avr8-gnu-toolchain/bin/../lib/gcc/avr/5.4.0/../../../../avr/lib/avrxmega6\libm.a(addsf3x.o) (__fp_inf)
c:/program files (x86)/atmel/studio/7.0/toolchain/avr8/avr8-gnu-toolchain/bin/../lib/gcc/avr/5.4.0/../../../../avr/lib/avrxmega6\libm.a(fp_nan.o)
                              c:/program files (x86)/atmel/studio/7.0/toolchain/avr8/avr8-gnu-toolchain/bin/../lib/gcc/avr/5.4.0/../../../../avr/lib/avrxmega6\libm.a(addsf3x.o) (__fp_nan)
c:/program files (x86)/atmel/studio/7.0/toolchain/avr8/avr8-gnu-toolchain/bin/../lib/gcc/avr/5.4.0/../../../../avr/lib/avrxmega6\libm.a(fp_pscA.o)
                              c:/program files (x86)/atmel/studio/7.0/toolchain/avr8/avr8-gnu-toolchain/bin/../lib/gcc/avr/5.4.0/../../../../avr/lib/avrxmega6\libm.a(addsf3x.o) (__fp_pscA)
c:/program files (x86)/atmel/studio/7.0/toolchain/avr8/avr8-gnu-toolchain/bin/../lib/gcc/avr/5.4.0/../../../../avr/lib/avrxmega6\libm.a(fp_pscB.o)
                              c:/program files (x86)/atmel/studio/7.0/toolchain/avr8/avr8-gnu-toolchain/bin/../lib/gcc/avr/5.4.0/../../../../avr/lib/avrxmega6\libm.a(addsf3x.o) (__fp_pscB)
c:/program files (x86)/atmel/studio/7.0/toolchain/avr8/avr8-gnu-toolchain/bin/../lib/gcc/avr/5.4.0/../../../../avr/lib/avrxmega6\libm.a(fp_round.o)
                              c:/program files (x86)/atmel/studio/7.0/toolchain/avr8/avr8-gnu-toolchain/bin/../lib/gcc/avr/5.4.0/../../../../avr/lib/avrxmega6\libm.a(addsf3.o) (__fp_round)
c:/program files (x86)/atmel/studio/7.0/toolchain/avr8/avr8-gnu-toolchain/bin/../lib/gcc/avr/5.4.0/../../../../avr/lib/avrxmega6\libm.a(fp_split3.o)
                              c:/program files (x86)/atmel/studio/7.0/toolchain/avr8/avr8-gnu-toolchain/bin/../lib/gcc/avr/5.4.0/../../../../avr/lib/avrxmega6\libm.a(addsf3x.o) (__fp_split3)
c:/program files (x86)/atmel/studio/7.0/toolchain/avr8/avr8-gnu-toolchain/bin/../lib/gcc/avr/5.4.0/../../../../avr/lib/avrxmega6\libm.a(fp_zero.o)
                              c:/program files (x86)/atmel/studio/7.0/toolchain/avr8/avr8-gnu-toolchain/bin/../lib/gcc/avr/5.4.0/../../../../avr/lib/avrxmega6\libm.a(addsf3x.o) (__fp_zero)
c:/program files (x86)/atmel/studio/7.0/toolchain/avr8/avr8-gnu-toolchain/bin/../lib/gcc/avr/5.4.0/../../../../avr/lib/avrxmega6\libm.a(log.o)
                              src/main.o (log)
c:/program files (x86)/atmel/studio/7.0/toolchain/avr8/avr8-gnu-toolchain/bin/../lib/gcc/avr/5.4.0/../../../../avr/lib/avrxmega6\libm.a(mulsf3.o)
                              src/adc_sensors/adc_sensors.o (__mulsf3)
c:/program files (x86)/atmel/studio/7.0/toolchain/avr8/avr8-gnu-toolchain/bin/../lib/gcc/avr/5.4.0/../../../../avr/lib/avrxmega6\libm.a(mulsf3x.o)
                              c:/program files (x86)/atmel/studio/7.0/toolchain/avr8/avr8-gnu-toolchain/bin/../lib/gcc/avr/5.4.0/../../../../avr/lib/avrxmega6\libm.a(log.o) (__mulsf3x)
c:/program files (x86)/atmel/studio/7.0/toolchain/avr8/avr8-gnu-toolchain/bin/../lib/gcc/avr/5.4.0/../../../../avr/lib/avrxmega6\libm.a(pow.o)
                              src/main.o (pow)
c:/program files (x86)/atmel/studio/7.0/toolchain/avr8/avr8-gnu-toolchain/bin/../lib/gcc/avr/5.4.0/../../../../avr/lib/avrxmega6\libm.a(exp.o)
                              c:/program files (x86)/atmel/studio/7.0/toolchain/avr8/avr8-gnu-toolchain/bin/../lib/gcc/avr/5.4.0/../../../../avr/lib/avrxmega6\libm.a(pow.o) (exp)
c:/program files (x86)/atmel/studio/7.0/toolchain/avr8/avr8-gnu-toolchain/bin/../lib/gcc/avr/5.4.0/../../../../avr/lib/avrxmega6\libm.a(fp_mpack.o)
                              c:/program files (x86)/atmel/studio/7.0/toolchain/avr8/avr8-gnu-toolchain/bin/../lib/gcc/avr/5.4.0/../../../../avr/lib/avrxmega6\libm.a(log.o) (__fp_mpack)
c:/program files (x86)/atmel/studio/7.0/toolchain/avr8/avr8-gnu-toolchain/bin/../lib/gcc/avr/5.4.0/../../../../avr/lib/avrxmega6\libm.a(fp_powser.o)
                              c:/program files (x86)/atmel/studio/7.0/toolchain/avr8/avr8-gnu-toolchain/bin/../lib/gcc/avr/5.4.0/../../../../avr/lib/avrxmega6\libm.a(log.o) (__fp_powser)
c:/program files (x86)/atmel/studio/7.0/toolchain/avr8/avr8-gnu-toolchain/bin/../lib/gcc/avr/5.4.0/../../../../avr/lib/avrxmega6\libm.a(inverse.o)
                              c:/program files (x86)/atmel/studio/7.0/toolchain/avr8/avr8-gnu-toolchain/bin/../lib/gcc/avr/5.4.0/../../../../avr/lib/avrxmega6\libm.a(exp.o) (inverse)
c:/program files (x86)/atmel/studio/7.0/toolchain/avr8/avr8-gnu-toolchain/bin/../lib/gcc/avr/5.4.0/../../../../avr/lib/avrxmega6\libm.a(ldexp.o)
                              c:/program files (x86)/atmel/studio/7.0/toolchain/avr8/avr8-gnu-toolchain/bin/../lib/gcc/avr/5.4.0/../../../../avr/lib/avrxmega6\libm.a(exp.o) (ldexp)
c:/program files (x86)/atmel/studio/7.0/toolchain/avr8/avr8-gnu-toolchain/bin/../lib/gcc/avr/5.4.0/../../../../avr/lib/avrxmega6\libm.a(modf.o)
                              c:/program files (x86)/atmel/studio/7.0/toolchain/avr8/avr8-gnu-toolchain/bin/../lib/gcc/avr/5.4.0/../../../../avr/lib/avrxmega6\libm.a(exp.o) (modf)
c:/program files (x86)/atmel/studio/7.0/toolchain/avr8/avr8-gnu-toolchain/bin/../lib/gcc/avr/5.4.0/avrxmega6\libgcc.a(_udivmodsi4.o)
                              src/ASF/xmega/drivers/usart/usart.o (__udivmodsi4)
c:/program files (x86)/atmel/studio/7.0/toolchain/avr8/avr8-gnu-toolchain/bin/../lib/gcc/avr/5.4.0/avrxmega6\libgcc.a(_exit.o)
                              C:/Program Files (x86)/Atmel/Studio/7.0/Packs/atmel/XMEGAA_DFP/1.3.146/gcc/dev/atxmega256a3bu/avrxmega6/crtatxmega256a3bu.o (exit)
c:/program files (x86)/atmel/studio/7.0/toolchain/avr8/avr8-gnu-toolchain/bin/../lib/gcc/avr/5.4.0/avrxmega6\libgcc.a(_copy_data.o)
                              src/ASF/common/services/sleepmgr/xmega/sleepmgr.o (__do_copy_data)
c:/program files (x86)/atmel/studio/7.0/toolchain/avr8/avr8-gnu-toolchain/bin/../lib/gcc/avr/5.4.0/avrxmega6\libgcc.a(_clear_bss.o)
                              src/adc_sensors/adc_sensors.o (__do_clear_bss)
c:/program files (x86)/atmel/studio/7.0/toolchain/avr8/avr8-gnu-toolchain/bin/../lib/gcc/avr/5.4.0/../../../../avr/lib/avrxmega6\libc.a(memcpy.o)
                              src/ASF/xmega/drivers/nvm/nvm.o (memcpy)
c:/program files (x86)/atmel/studio/7.0/toolchain/avr8/avr8-gnu-toolchain/bin/../lib/gcc/avr/5.4.0/../../../../avr/lib/avrxmega6\libc.a(snprintf.o)
                              src/main.o (snprintf)
c:/program files (x86)/atmel/studio/7.0/toolchain/avr8/avr8-gnu-toolchain/bin/../lib/gcc/avr/5.4.0/../../../../avr/lib/avrxmega6\libc.a(vfprintf_std.o)
                              c:/program files (x86)/atmel/studio/7.0/toolchain/avr8/avr8-gnu-toolchain/bin/../lib/gcc/avr/5.4.0/../../../../avr/lib/avrxmega6\libc.a(snprintf.o) (vfprintf)
c:/program files (x86)/atmel/studio/7.0/toolchain/avr8/avr8-gnu-toolchain/bin/../lib/gcc/avr/5.4.0/../../../../avr/lib/avrxmega6\libc.a(strnlen_P.o)
                              c:/program files (x86)/atmel/studio/7.0/toolchain/avr8/avr8-gnu-toolchain/bin/../lib/gcc/avr/5.4.0/../../../../avr/lib/avrxmega6\libc.a(vfprintf_std.o) (strnlen_P)
c:/program files (x86)/atmel/studio/7.0/toolchain/avr8/avr8-gnu-toolchain/bin/../lib/gcc/avr/5.4.0/../../../../avr/lib/avrxmega6\libc.a(strnlen.o)
                              c:/program files (x86)/atmel/studio/7.0/toolchain/avr8/avr8-gnu-toolchain/bin/../lib/gcc/avr/5.4.0/../../../../avr/lib/avrxmega6\libc.a(vfprintf_std.o) (strnlen)
c:/program files (x86)/atmel/studio/7.0/toolchain/avr8/avr8-gnu-toolchain/bin/../lib/gcc/avr/5.4.0/../../../../avr/lib/avrxmega6\libc.a(fputc.o)
                              c:/program files (x86)/atmel/studio/7.0/toolchain/avr8/avr8-gnu-toolchain/bin/../lib/gcc/avr/5.4.0/../../../../avr/lib/avrxmega6\libc.a(vfprintf_std.o) (fputc)
c:/program files (x86)/atmel/studio/7.0/toolchain/avr8/avr8-gnu-toolchain/bin/../lib/gcc/avr/5.4.0/../../../../avr/lib/avrxmega6\libc.a(ultoa_invert.o)
                              c:/program files (x86)/atmel/studio/7.0/toolchain/avr8/avr8-gnu-toolchain/bin/../lib/gcc/avr/5.4.0/../../../../avr/lib/avrxmega6\libc.a(vfprintf_std.o) (__ultoa_invert)

Allocating common symbols
Common symbol       size              file

adcb_callback       0x2               src/ASF/xmega/drivers/adc/adc.o
sleepmgr_locks      0x6               src/ASF/common/services/sleepmgr/xmega/sleepmgr.o
adca_callback       0x2               src/ASF/xmega/drivers/adc/adc.o

Discarded input sections

 .data          0x00000000        0x0 C:/Program Files (x86)/Atmel/Studio/7.0/Packs/atmel/XMEGAA_DFP/1.3.146/gcc/dev/atxmega256a3bu/avrxmega6/crtatxmega256a3bu.o
 .bss           0x00000000        0x0 C:/Program Files (x86)/Atmel/Studio/7.0/Packs/atmel/XMEGAA_DFP/1.3.146/gcc/dev/atxmega256a3bu/avrxmega6/crtatxmega256a3bu.o
 .group         0x00000000        0x8 src/adc_sensors/adc_sensors.o
 .group         0x00000000        0x8 src/adc_sensors/adc_sensors.o
 .group         0x00000000        0x8 src/adc_sensors/adc_sensors.o
 .group         0x00000000        0x8 src/adc_sensors/adc_sensors.o
 .group         0x00000000        0x8 src/adc_sensors/adc_sensors.o
 .group         0x00000000        0x8 src/adc_sensors/adc_sensors.o
 .group         0x00000000        0x8 src/adc_sensors/adc_sensors.o
 .group         0x00000000        0x8 src/adc_sensors/adc_sensors.o
 .group         0x00000000        0x8 src/adc_sensors/adc_sensors.o
 .group         0x00000000        0x8 src/adc_sensors/adc_sensors.o
 .group         0x00000000        0x8 src/adc_sensors/adc_sensors.o
 .group         0x00000000        0x8 src/adc_sensors/adc_sensors.o
 .group         0x00000000        0x8 src/adc_sensors/adc_sensors.o
 .group         0x00000000        0x8 src/adc_sensors/adc_sensors.o
 .group         0x00000000        0x8 src/adc_sensors/adc_sensors.o
 .group         0x00000000        0x8 src/adc_sensors/adc_sensors.o
Memory Configuration

Name             Origin             Length             Attributes
text             0x00000000         0x00042000         xr
data             0x00802000         0x00004000         rw !x
eeprom           0x00810000         0x00001000         rw !x
fuse             0x00820000         0x00000006         rw !x
lock             0x00830000         0x00000400         rw !x
signature        0x00840000         0x00000400         rw !x
user_signatures  0x00850000         0x00000400         rw !x
*default*        0x00000000         0xffffffff

Linker script and memory map

LOAD C:/Program Files (x86)/Atmel/Studio/7.0/Packs/atmel/XMEGAA_DFP/1.3.146/gcc/dev/atxmega256a3bu/avrxmega6/crtatxmega256a3bu.o
LOAD src/adc_sensors/adc_sensors.o
LOAD src/ASF/common/components/display/st7565r/st7565r.o
LOAD src/ASF/common/services/gfx_mono/gfx_mono_c12832_a1z.o
LOAD src/ASF/xmega/drivers/adc/adc.o
LOAD src/ASF/xmega/drivers/usart/usart.o
LOAD src/ASF/xmega/drivers/adc/xmega_aau/adc_aau.o
LOAD src/ASF/common/services/spi/xmega_usart_spi/usart_spi.o
LOAD src/ASF/common/services/spi/xmega_spi/spi_master.o
LOAD src/ASF/common/services/sleepmgr/xmega/sleepmgr.o
LOAD src/ASF/common/services/gfx_mono/gfx_mono_framebuffer.o
LOAD src/ASF/common/services/gfx_mono/gfx_mono_generic.o
LOAD src/ASF/common/services/clock/xmega/sysclk.o
LOAD src/ASF/common/services/gfx_mono/gfx_mono_menu.o
LOAD src/ASF/xmega/drivers/nvm/nvm.o
LOAD src/ASF/xmega/drivers/spi/spi.o
LOAD src/ASF/xmega/drivers/nvm/nvm_asm.o
LOAD src/ASF/xmega/drivers/cpu/ccp.o
LOAD src/ASF/common/services/gfx_mono/gfx_mono_text.o
LOAD src/ASF/common/services/gfx_mono/sysfont.o
LOAD src/ASF/common/services/ioport/xmega/ioport_compat.o
LOAD src/ASF/xmega/boards/xmega_a3bu_xplained/init.o
LOAD src/main.o
START GROUP
LOAD c:/program files (x86)/atmel/studio/7.0/toolchain/avr8/avr8-gnu-toolchain/bin/../lib/gcc/avr/5.4.0/../../../../avr/lib/avrxmega6\libm.a
END GROUP
Address of section .BOOT set to 0x40000
START GROUP
LOAD c:/program files (x86)/atmel/studio/7.0/toolchain/avr8/avr8-gnu-toolchain/bin/../lib/gcc/avr/5.4.0/avrxmega6\libgcc.a
LOAD c:/program files (x86)/atmel/studio/7.0/toolchain/avr8/avr8-gnu-toolchain/bin/../lib/gcc/avr/5.4.0/../../../../avr/lib/avrxmega6\libm.a
LOAD c:/program files (x86)/atmel/studio/7.0/toolchain/avr8/avr8-gnu-toolchain/bin/../lib/gcc/avr/5.4.0/../../../../avr/lib/avrxmega6\libc.a
LOAD C:/Program Files (x86)/Atmel/Studio/7.0/Packs/atmel/XMEGAA_DFP/1.3.146/gcc/dev/atxmega256a3bu/avrxmega6\libatxmega256a3bu.a
END GROUP
                [0x00000000]                __TEXT_REGION_ORIGIN__ = DEFINED (__TEXT_REGION_ORIGIN__)?__TEXT_REGION_ORIGIN__:0x0
                [0x00802000]                __DATA_REGION_ORIGIN__ = DEFINED (__DATA_REGION_ORIGIN__)?__DATA_REGION_ORIGIN__:0x802000
                [0x00042000]                __TEXT_REGION_LENGTH__ = DEFINED (__TEXT_REGION_LENGTH__)?__TEXT_REGION_LENGTH__:0x100000
                [0x00004000]                __DATA_REGION_LENGTH__ = DEFINED (__DATA_REGION_LENGTH__)?__DATA_REGION_LENGTH__:0xffa0
                [0x00001000]                __EEPROM_REGION_LENGTH__ = DEFINED (__EEPROM_REGION_LENGTH__)?__EEPROM_REGION_LENGTH__:0x10000
                [0x00000006]                __FUSE_REGION_LENGTH__ = DEFINED (__FUSE_REGION_LENGTH__)?__FUSE_REGION_LENGTH__:0x400
                0x00000400                __LOCK_REGION_LENGTH__ = DEFINED (__LOCK_REGION_LENGTH__)?__LOCK_REGION_LENGTH__:0x400
                0x00000400                __SIGNATURE_REGION_LENGTH__ = DEFINED (__SIGNATURE_REGION_LENGTH__)?__SIGNATURE_REGION_LENGTH__:0x400
                0x00000400                __USER_SIGNATURE_REGION_LENGTH__ = DEFINED (__USER_SIGNATURE_REGION_LENGTH__)?__USER_SIGNATURE_REGION_LENGTH__:0x400

.hash
 *(.hash)

.dynsym
 *(.dynsym)

.dynstr
 *(.dynstr)

.gnu.version
 *(.gnu.version)

.gnu.version_d
 *(.gnu.version_d)

.gnu.version_r
 *(.gnu.version_r)

.rel.init
 *(.rel.init)

.rela.init
 *(.rela.init)

.rel.text
 *(.rel.text)
 *(.rel.text.*)
 *(.rel.gnu.linkonce.t*)

.rela.text
 *(.rela.text)
 *(.rela.text.*)
 *(.rela.gnu.linkonce.t*)

.rel.fini
 *(.rel.fini)

.rela.fini
 *(.rela.fini)

.rel.rodata
 *(.rel.rodata)
 *(.rel.rodata.*)
 *(.rel.gnu.linkonce.r*)

.rela.rodata
 *(.rela.rodata)
 *(.rela.rodata.*)
 *(.rela.gnu.linkonce.r*)

.rel.data
 *(.rel.data)
 *(.rel.data.*)
 *(.rel.gnu.linkonce.d*)

.rela.data
 *(.rela.data)
 *(.rela.data.*)
 *(.rela.gnu.linkonce.d*)

.rel.ctors
 *(.rel.ctors)

.rela.ctors
 *(.rela.ctors)

.rel.dtors
 *(.rel.dtors)

.rela.dtors
 *(.rela.dtors)

.rel.got
 *(.rel.got)

.rela.got
 *(.rela.got)

.rel.bss
 *(.rel.bss)

.rela.bss
 *(.rela.bss)

.rel.plt
 *(.rel.plt)

.rela.plt
 *(.rela.plt)

.text           0x00000000     0x2de4
 *(.vectors)
 .vectors       0x00000000      0x1fc C:/Program Files (x86)/Atmel/Studio/7.0/Packs/atmel/XMEGAA_DFP/1.3.146/gcc/dev/atxmega256a3bu/avrxmega6/crtatxmega256a3bu.o
                0x00000000                __vector_default
                0x00000000                __vectors
 *(.vectors)
 *(.progmem.gcc*)
 .progmem.gcc_fplib
                0x000001fc       0x5a c:/program files (x86)/atmel/studio/7.0/toolchain/avr8/avr8-gnu-toolchain/bin/../lib/gcc/avr/5.4.0/../../../../avr/lib/avrxmega6\libm.a(log.o)
 .progmem.gcc_fplib
                0x00000256       0x28 c:/program files (x86)/atmel/studio/7.0/toolchain/avr8/avr8-gnu-toolchain/bin/../lib/gcc/avr/5.4.0/../../../../avr/lib/avrxmega6\libm.a(exp.o)
                0x0000027e                . = ALIGN (0x2)
                0x0000027e                __trampolines_start = .
 *(.trampolines)
 .trampolines   0x0000027e        0x0 linker stubs
 *(.trampolines*)
                0x0000027e                __trampolines_end = .
 *libprintf_flt.a:*(.progmem.data)
 *libc.a:*(.progmem.data)
 *(.progmem*)
 .progmem.data.sysfont_glyphs
                0x0000027e      0x292 src/ASF/common/services/gfx_mono/sysfont.o
                0x00000510                . = ALIGN (0x2)
 *(.jumptables)
 *(.jumptables*)
 *(.lowtext)
 *(.lowtext*)
                0x00000510                __ctors_start = .
 *(.ctors)
                0x00000510                __ctors_end = .
                0x00000510                __dtors_start = .
 *(.dtors)
                0x00000510                __dtors_end = .
 SORT(*)(.ctors)
 SORT(*)(.dtors)
 *(.init0)
 .init0         0x00000510        0x0 C:/Program Files (x86)/Atmel/Studio/7.0/Packs/atmel/XMEGAA_DFP/1.3.146/gcc/dev/atxmega256a3bu/avrxmega6/crtatxmega256a3bu.o
                0x00000510                __init
 *(.init0)
 *(.init1)
 *(.init1)
 *(.init2)
 .init2         0x00000510       0x10 C:/Program Files (x86)/Atmel/Studio/7.0/Packs/atmel/XMEGAA_DFP/1.3.146/gcc/dev/atxmega256a3bu/avrxmega6/crtatxmega256a3bu.o
 *(.init2)
 *(.init3)
 *(.init3)
 *(.init4)
 .init4         0x00000520       0x1a c:/program files (x86)/atmel/studio/7.0/toolchain/avr8/avr8-gnu-toolchain/bin/../lib/gcc/avr/5.4.0/avrxmega6\libgcc.a(_copy_data.o)
                0x00000520                __do_copy_data
 .init4         0x0000053a       0x10 c:/program files (x86)/atmel/studio/7.0/toolchain/avr8/avr8-gnu-toolchain/bin/../lib/gcc/avr/5.4.0/avrxmega6\libgcc.a(_clear_bss.o)
                0x0000053a                __do_clear_bss
 *(.init4)
 *(.init5)
 *(.init5)
 *(.init6)
 *(.init6)
 *(.init7)
 *(.init7)
 *(.init8)
 *(.init8)
 *(.init9)
 .init9         0x0000054a        0x8 C:/Program Files (x86)/Atmel/Studio/7.0/Packs/atmel/XMEGAA_DFP/1.3.146/gcc/dev/atxmega256a3bu/avrxmega6/crtatxmega256a3bu.o
 *(.init9)
 *(.text)
 .text          0x00000552        0x2 C:/Program Files (x86)/Atmel/Studio/7.0/Packs/atmel/XMEGAA_DFP/1.3.146/gcc/dev/atxmega256a3bu/avrxmega6/crtatxmega256a3bu.o
                0x00000552                __vector_38
                0x00000552                __vector_104
                0x00000552                __vector_22
                0x00000552                __vector_63
                0x00000552                __vector_28
                0x00000552                __vector_67
                0x00000552                __vector_1
                0x00000552                __vector_119
                0x00000552                __vector_32
                0x00000552                __vector_75
                0x00000552                __vector_91
                0x00000552                __vector_34
                0x00000552                __vector_62
                0x00000552                __vector_77
                0x00000552                __vector_102
                0x00000552                __vector_24
                0x00000552                __vector_12
                0x00000552                __vector_55
                0x00000552                __vector_69
                0x00000552                __vector_81
                0x00000552                __vector_90
                0x00000552                __vector_46
                0x00000552                __bad_interrupt
                0x00000552                __vector_122
                0x00000552                __vector_114
                0x00000552                __vector_6
                0x00000552                __vector_110
                0x00000552                __vector_31
                0x00000552                __vector_92
                0x00000552                __vector_35
                0x00000552                __vector_78
                0x00000552                __vector_117
                0x00000552                __vector_107
                0x00000552                __vector_3
                0x00000552                __vector_105
                0x00000552                __vector_98
                0x00000552                __vector_23
                0x00000552                __vector_68
                0x00000552                __vector_30
                0x00000552                __vector_45
                0x00000552                __vector_25
                0x00000552                __vector_93
                0x00000552                __vector_61
                0x00000552                __vector_11
                0x00000552                __vector_54
                0x00000552                __vector_99
                0x00000552                __vector_13
                0x00000552                __vector_17
                0x00000552                __vector_19
                0x00000552                __vector_56
                0x00000552                __vector_7
                0x00000552                __vector_125
                0x00000552                __vector_49
                0x00000552                __vector_123
                0x00000552                __vector_86
                0x00000552                __vector_100
                0x00000552                __vector_101
                0x00000552                __vector_64
                0x00000552                __vector_88
                0x00000552                __vector_109
                0x00000552                __vector_43
                0x00000552                __vector_27
                0x00000552                __vector_5
                0x00000552                __vector_113
                0x00000552                __vector_33
                0x00000552                __vector_76
                0x00000552                __vector_115
                0x00000552                __vector_47
                0x00000552                __vector_52
                0x00000552                __vector_37
                0x00000552                __vector_95
                0x00000552                __vector_103
                0x00000552                __vector_96
                0x00000552                __vector_89
                0x00000552                __vector_108
                0x00000552                __vector_4
                0x00000552                __vector_44
                0x00000552                __vector_82
                0x00000552                __vector_106
                0x00000552                __vector_118
                0x00000552                __vector_51
                0x00000552                __vector_9
                0x00000552                __vector_2
                0x00000552                __vector_21
                0x00000552                __vector_15
                0x00000552                __vector_66
                0x00000552                __vector_36
                0x00000552                __vector_79
                0x00000552                __vector_58
                0x00000552                __vector_70
                0x00000552                __vector_83
                0x00000552                __vector_29
                0x00000552                __vector_60
                0x00000552                __vector_121
                0x00000552                __vector_85
                0x00000552                __vector_94
                0x00000552                __vector_126
                0x00000552                __vector_8
                0x00000552                __vector_26
                0x00000552                __vector_48
                0x00000552                __vector_124
                0x00000552                __vector_116
                0x00000552                __vector_112
                0x00000552                __vector_111
                0x00000552                __vector_80
                0x00000552                __vector_14
                0x00000552                __vector_84
                0x00000552                __vector_57
                0x00000552                __vector_53
                0x00000552                __vector_10
                0x00000552                __vector_50
                0x00000552                __vector_16
                0x00000552                __vector_59
                0x00000552                __vector_18
                0x00000552                __vector_97
                0x00000552                __vector_20
                0x00000552                __vector_87
                0x00000552                __vector_65
                0x00000552                __vector_120
                0x00000554                . = ALIGN (0x2)
 *(.text.*)
 .text.adc_handler
                0x00000554       0xd0 src/adc_sensors/adc_sensors.o
                0x00000554                adc_handler
 .text.ntc_data_is_ready
                0x00000624       0x2c src/adc_sensors/adc_sensors.o
                0x00000624                ntc_data_is_ready
 .text.adc_sensors_init
                0x00000650       0x9e src/adc_sensors/adc_sensors.o
                0x00000650                adc_sensors_init
 .text.ntc_get_temperature
                0x000006ee       0x60 src/adc_sensors/adc_sensors.o
                0x000006ee                ntc_get_temperature
 .text.__portable_avr_delay_cycles
                0x0000074e       0x16 src/ASF/common/components/display/st7565r/st7565r.o
 .text.st7565r_init
                0x00000764      0x398 src/ASF/common/components/display/st7565r/st7565r.o
                0x00000764                st7565r_init
 .text.gfx_mono_st7565r_put_byte
                0x00000afc      0x14e src/ASF/common/services/gfx_mono/gfx_mono_c12832_a1z.o
                0x00000afc                gfx_mono_st7565r_put_byte
 .text.gfx_mono_st7565r_init
                0x00000c4a       0x84 src/ASF/common/services/gfx_mono/gfx_mono_c12832_a1z.o
                0x00000c4a                gfx_mono_st7565r_init
 .text.gfx_mono_st7565r_draw_pixel
                0x00000cce       0x6c src/ASF/common/services/gfx_mono/gfx_mono_c12832_a1z.o
                0x00000cce                gfx_mono_st7565r_draw_pixel
 .text.gfx_mono_st7565r_get_byte
                0x00000d3a        0x4 src/ASF/common/services/gfx_mono/gfx_mono_c12832_a1z.o
                0x00000d3a                gfx_mono_st7565r_get_byte
 .text.adc_set_callback
                0x00000d3e       0x40 src/ASF/xmega/drivers/adc/adc.o
                0x00000d3e                adc_set_callback
 .text.adc_enable_clock
                0x00000d7e       0x3e src/ASF/xmega/drivers/adc/adc.o
                0x00000d7e                adc_enable_clock
 .text.adc_disable_clock
                0x00000dbc       0x3a src/ASF/xmega/drivers/adc/adc.o
                0x00000dbc                adc_disable_clock
 .text.adc_enable
                0x00000df6       0x58 src/ASF/xmega/drivers/adc/adc.o
                0x00000df6                adc_enable
 .text.usart_spi_set_baudrate
                0x00000e4e       0x64 src/ASF/xmega/drivers/usart/usart.o
                0x00000e4e                usart_spi_set_baudrate
 .text.usart_init_spi
                0x00000eb2      0x3c8 src/ASF/xmega/drivers/usart/usart.o
                0x00000eb2                usart_init_spi
 .text.__vector_71
                0x0000127a       0x64 src/ASF/xmega/drivers/adc/xmega_aau/adc_aau.o
                0x0000127a                __vector_71
 .text.__vector_72
                0x000012de       0x64 src/ASF/xmega/drivers/adc/xmega_aau/adc_aau.o
                0x000012de                __vector_72
 .text.__vector_73
                0x00001342       0x64 src/ASF/xmega/drivers/adc/xmega_aau/adc_aau.o
                0x00001342                __vector_73
 .text.__vector_74
                0x000013a6       0x64 src/ASF/xmega/drivers/adc/xmega_aau/adc_aau.o
                0x000013a6                __vector_74
 .text.__vector_39
                0x0000140a       0x64 src/ASF/xmega/drivers/adc/xmega_aau/adc_aau.o
                0x0000140a                __vector_39
 .text.__vector_40
                0x0000146e       0x64 src/ASF/xmega/drivers/adc/xmega_aau/adc_aau.o
                0x0000146e                __vector_40
 .text.__vector_41
                0x000014d2       0x64 src/ASF/xmega/drivers/adc/xmega_aau/adc_aau.o
                0x000014d2                __vector_41
 .text.__vector_42
                0x00001536       0x64 src/ASF/xmega/drivers/adc/xmega_aau/adc_aau.o
                0x00001536                __vector_42
 .text.adc_write_configuration
                0x0000159a       0xcc src/ASF/xmega/drivers/adc/xmega_aau/adc_aau.o
                0x0000159a                adc_write_configuration
 .text.adc_read_configuration
                0x00001666       0x72 src/ASF/xmega/drivers/adc/xmega_aau/adc_aau.o
                0x00001666                adc_read_configuration
 .text.adcch_write_configuration
                0x000016d8       0x96 src/ASF/xmega/drivers/adc/xmega_aau/adc_aau.o
                0x000016d8                adcch_write_configuration
 .text.adcch_read_configuration
                0x0000176e       0x96 src/ASF/xmega/drivers/adc/xmega_aau/adc_aau.o
                0x0000176e                adcch_read_configuration
 .text.usart_spi_init
                0x00001804       0x5e src/ASF/common/services/spi/xmega_usart_spi/usart_spi.o
                0x00001804                usart_spi_init
 .text.usart_spi_setup_device
                0x00001862       0x34 src/ASF/common/services/spi/xmega_usart_spi/usart_spi.o
                0x00001862                usart_spi_setup_device
 .text.usart_spi_select_device
                0x00001896       0x2c src/ASF/common/services/spi/xmega_usart_spi/usart_spi.o
                0x00001896                usart_spi_select_device
 .text.usart_spi_deselect_device
                0x000018c2       0x2c src/ASF/common/services/spi/xmega_usart_spi/usart_spi.o
                0x000018c2                usart_spi_deselect_device
 .text.gfx_mono_set_framebuffer
                0x000018ee        0xa src/ASF/common/services/gfx_mono/gfx_mono_framebuffer.o
                0x000018ee                gfx_mono_set_framebuffer
 .text.gfx_mono_framebuffer_put_byte
                0x000018f8       0x1c src/ASF/common/services/gfx_mono/gfx_mono_framebuffer.o
                0x000018f8                gfx_mono_framebuffer_put_byte
 .text.gfx_mono_framebuffer_get_byte
                0x00001914       0x1c src/ASF/common/services/gfx_mono/gfx_mono_framebuffer.o
                0x00001914                gfx_mono_framebuffer_get_byte
 .text.gfx_mono_generic_draw_horizontal_line
                0x00001930       0xc4 src/ASF/common/services/gfx_mono/gfx_mono_generic.o
                0x00001930                gfx_mono_generic_draw_horizontal_line
 .text.gfx_mono_generic_draw_filled_rect
                0x000019f4       0x34 src/ASF/common/services/gfx_mono/gfx_mono_generic.o
                0x000019f4                gfx_mono_generic_draw_filled_rect
 .text.sysclk_enable_module
                0x00001a28       0x2c src/ASF/common/services/clock/xmega/sysclk.o
                0x00001a28                sysclk_enable_module
 .text.sysclk_disable_module
                0x00001a54       0x2a src/ASF/common/services/clock/xmega/sysclk.o
                0x00001a54                sysclk_disable_module
 .text.nvm_read_byte
                0x00001a7e       0x14 src/ASF/xmega/drivers/nvm/nvm_asm.o
                0x00001a7e                nvm_read_byte
 .text.gfx_mono_draw_char
                0x00001a92       0xba src/ASF/common/services/gfx_mono/gfx_mono_text.o
                0x00001a92                gfx_mono_draw_char
 .text.gfx_mono_draw_string
                0x00001b4c       0x52 src/ASF/common/services/gfx_mono/gfx_mono_text.o
                0x00001b4c                gfx_mono_draw_string
 .text.ioport_configure_port_pin
                0x00001b9e       0x4e src/ASF/common/services/ioport/xmega/ioport_compat.o
                0x00001b9e                ioport_configure_port_pin
 .text.board_init
                0x00001bec      0x13a src/ASF/xmega/boards/xmega_a3bu_xplained/init.o
                0x00001bec                board_init
 .text.__portable_avr_delay_cycles
                0x00001d26       0x16 src/main.o
 .text.adc_read
                0x00001d3c       0x2a src/main.o
 .text.checkFire
                0x00001d66       0x20 src/main.o
                0x00001d66                checkFire
 .text.ResistanceCalculation
                0x00001d86       0x52 src/main.o
                0x00001d86                ResistanceCalculation
 .text.SensorCalibration
                0x00001dd8       0xea src/main.o
                0x00001dd8                SensorCalibration
 .text.ReadSensor
                0x00001ec2       0x5e src/main.o
                0x00001ec2                ReadSensor
 .text.GetPercentage
                0x00001f20       0x3e src/main.o
                0x00001f20                GetPercentage
 .text.main     0x00001f5e      0x1dc src/main.o
                0x00001f5e                main
 .text.avr-libc.fplib
                0x0000213a        0xa c:/program files (x86)/atmel/studio/7.0/toolchain/avr8/avr8-gnu-toolchain/bin/../lib/gcc/avr/5.4.0/../../../../avr/lib/avrxmega6\libm.a(addsf3.o)
                0x0000213a                __subsf3
                0x0000213c                __addsf3
 .text.avr-libc.fplib
                0x00002144       0xc0 c:/program files (x86)/atmel/studio/7.0/toolchain/avr8/avr8-gnu-toolchain/bin/../lib/gcc/avr/5.4.0/../../../../avr/lib/avrxmega6\libm.a(addsf3x.o)
                0x0000215e                __addsf3x
 .text.avr-libc.fplib
                0x00002204        0x4 c:/program files (x86)/atmel/studio/7.0/toolchain/avr8/avr8-gnu-toolchain/bin/../lib/gcc/avr/5.4.0/../../../../avr/lib/avrxmega6\libm.a(divsf3.o)
                0x00002204                __divsf3
 .text.avr-libc.fplib
                0x00002208       0xcc c:/program files (x86)/atmel/studio/7.0/toolchain/avr8/avr8-gnu-toolchain/bin/../lib/gcc/avr/5.4.0/../../../../avr/lib/avrxmega6\libm.a(divsf3x.o)
                0x0000221e                __divsf3x
                0x00002222                __divsf3_pse
 .text.avr-libc.fplib
                0x000022d4        0xa c:/program files (x86)/atmel/studio/7.0/toolchain/avr8/avr8-gnu-toolchain/bin/../lib/gcc/avr/5.4.0/../../../../avr/lib/avrxmega6\libm.a(fixsfsi.o)
                0x000022d4                __fixsfsi
 .text.avr-libc.fplib
                0x000022de       0x58 c:/program files (x86)/atmel/studio/7.0/toolchain/avr8/avr8-gnu-toolchain/bin/../lib/gcc/avr/5.4.0/../../../../avr/lib/avrxmega6\libm.a(fixunssfsi.o)
                0x000022de                __fixunssfsi
 .text.avr-libc.fplib
                0x00002336       0x7a c:/program files (x86)/atmel/studio/7.0/toolchain/avr8/avr8-gnu-toolchain/bin/../lib/gcc/avr/5.4.0/../../../../avr/lib/avrxmega6\libm.a(floatsisf.o)
                0x00002336                __floatunsisf
                0x0000233a                __floatsisf
 .text.avr-libc.fplib
                0x000023b0        0xc c:/program files (x86)/atmel/studio/7.0/toolchain/avr8/avr8-gnu-toolchain/bin/../lib/gcc/avr/5.4.0/../../../../avr/lib/avrxmega6\libm.a(fp_inf.o)
                0x000023b0                __fp_inf
 .text.avr-libc.fplib
                0x000023bc        0x6 c:/program files (x86)/atmel/studio/7.0/toolchain/avr8/avr8-gnu-toolchain/bin/../lib/gcc/avr/5.4.0/../../../../avr/lib/avrxmega6\libm.a(fp_nan.o)
                0x000023bc                __fp_nan
 .text.avr-libc.fplib
                0x000023c2        0xe c:/program files (x86)/atmel/studio/7.0/toolchain/avr8/avr8-gnu-toolchain/bin/../lib/gcc/avr/5.4.0/../../../../avr/lib/avrxmega6\libm.a(fp_pscA.o)
                0x000023c2                __fp_pscA
 .text.avr-libc.fplib
                0x000023d0        0xe c:/program files (x86)/atmel/studio/7.0/toolchain/avr8/avr8-gnu-toolchain/bin/../lib/gcc/avr/5.4.0/../../../../avr/lib/avrxmega6\libm.a(fp_pscB.o)
                0x000023d0                __fp_pscB
 .text.avr-libc.fplib
                0x000023de       0x22 c:/program files (x86)/atmel/studio/7.0/toolchain/avr8/avr8-gnu-toolchain/bin/../lib/gcc/avr/5.4.0/../../../../avr/lib/avrxmega6\libm.a(fp_round.o)
                0x000023de                __fp_round
 .text.avr-libc.fplib
                0x00002400       0x44 c:/program files (x86)/atmel/studio/7.0/toolchain/avr8/avr8-gnu-toolchain/bin/../lib/gcc/avr/5.4.0/../../../../avr/lib/avrxmega6\libm.a(fp_split3.o)
                0x00002400                __fp_split3
                0x00002410                __fp_splitA
 .text.avr-libc.fplib
                0x00002444        0xe c:/program files (x86)/atmel/studio/7.0/toolchain/avr8/avr8-gnu-toolchain/bin/../lib/gcc/avr/5.4.0/../../../../avr/lib/avrxmega6\libm.a(fp_zero.o)
                0x00002444                __fp_zero
                0x00002446                __fp_szero
 .text.avr-libc.fplib
                0x00002452       0x8a c:/program files (x86)/atmel/studio/7.0/toolchain/avr8/avr8-gnu-toolchain/bin/../lib/gcc/avr/5.4.0/../../../../avr/lib/avrxmega6\libm.a(log.o)
                0x0000245c                log
 .text.avr-libc.fplib
                0x000024dc        0x4 c:/program files (x86)/atmel/studio/7.0/toolchain/avr8/avr8-gnu-toolchain/bin/../lib/gcc/avr/5.4.0/../../../../avr/lib/avrxmega6\libm.a(mulsf3.o)
                0x000024dc                __mulsf3
 .text.avr-libc.fplib
                0x000024e0       0xc2 c:/program files (x86)/atmel/studio/7.0/toolchain/avr8/avr8-gnu-toolchain/bin/../lib/gcc/avr/5.4.0/../../../../avr/lib/avrxmega6\libm.a(mulsf3x.o)
                0x000024f4                __mulsf3x
                0x000024f8                __mulsf3_pse
 .text.avr-libc.fplib
                0x000025a2       0x98 c:/program files (x86)/atmel/studio/7.0/toolchain/avr8/avr8-gnu-toolchain/bin/../lib/gcc/avr/5.4.0/../../../../avr/lib/avrxmega6\libm.a(pow.o)
                0x000025a2                pow
 .text.avr-libc.fplib
                0x0000263a       0x62 c:/program files (x86)/atmel/studio/7.0/toolchain/avr8/avr8-gnu-toolchain/bin/../lib/gcc/avr/5.4.0/../../../../avr/lib/avrxmega6\libm.a(exp.o)
                0x00002644                exp
 .text.avr-libc.fplib
                0x0000269c       0x1c c:/program files (x86)/atmel/studio/7.0/toolchain/avr8/avr8-gnu-toolchain/bin/../lib/gcc/avr/5.4.0/../../../../avr/lib/avrxmega6\libm.a(fp_mpack.o)
                0x0000269c                __fp_mpack
                0x000026a0                __fp_mpack_finite
 .text.avr-libc.fplib
                0x000026b8       0x4a c:/program files (x86)/atmel/studio/7.0/toolchain/avr8/avr8-gnu-toolchain/bin/../lib/gcc/avr/5.4.0/../../../../avr/lib/avrxmega6\libm.a(fp_powser.o)
                0x000026b8                __fp_powser
 .text.avr-libc.fplib
                0x00002702        0xe c:/program files (x86)/atmel/studio/7.0/toolchain/avr8/avr8-gnu-toolchain/bin/../lib/gcc/avr/5.4.0/../../../../avr/lib/avrxmega6\libm.a(inverse.o)
                0x00002702                inverse
 .text.avr-libc.fplib
                0x00002710       0x6c c:/program files (x86)/atmel/studio/7.0/toolchain/avr8/avr8-gnu-toolchain/bin/../lib/gcc/avr/5.4.0/../../../../avr/lib/avrxmega6\libm.a(ldexp.o)
                0x00002714                ldexp
 .text.avr-libc.fplib
                0x0000277c       0x66 c:/program files (x86)/atmel/studio/7.0/toolchain/avr8/avr8-gnu-toolchain/bin/../lib/gcc/avr/5.4.0/../../../../avr/lib/avrxmega6\libm.a(modf.o)
                0x0000277c                modf
                0x0000277c                modff
 .text.libgcc.div
                0x000027e2       0x44 c:/program files (x86)/atmel/studio/7.0/toolchain/avr8/avr8-gnu-toolchain/bin/../lib/gcc/avr/5.4.0/avrxmega6\libgcc.a(_udivmodsi4.o)
                0x000027e2                __udivmodsi4
 .text.avr-libc
                0x00002826       0x6c c:/program files (x86)/atmel/studio/7.0/toolchain/avr8/avr8-gnu-toolchain/bin/../lib/gcc/avr/5.4.0/../../../../avr/lib/avrxmega6\libc.a(snprintf.o)
                0x00002826                snprintf
 .text.avr-libc
                0x00002892      0x3ee c:/program files (x86)/atmel/studio/7.0/toolchain/avr8/avr8-gnu-toolchain/bin/../lib/gcc/avr/5.4.0/../../../../avr/lib/avrxmega6\libc.a(vfprintf_std.o)
                0x00002892                vfprintf
 .text.avr-libc
                0x00002c80       0x16 c:/program files (x86)/atmel/studio/7.0/toolchain/avr8/avr8-gnu-toolchain/bin/../lib/gcc/avr/5.4.0/../../../../avr/lib/avrxmega6\libc.a(strnlen_P.o)
                0x00002c80                strnlen_P
 .text.avr-libc
                0x00002c96       0x16 c:/program files (x86)/atmel/studio/7.0/toolchain/avr8/avr8-gnu-toolchain/bin/../lib/gcc/avr/5.4.0/../../../../avr/lib/avrxmega6\libc.a(strnlen.o)
                0x00002c96                strnlen
 .text.avr-libc
                0x00002cac       0x78 c:/program files (x86)/atmel/studio/7.0/toolchain/avr8/avr8-gnu-toolchain/bin/../lib/gcc/avr/5.4.0/../../../../avr/lib/avrxmega6\libc.a(fputc.o)
                0x00002cac                fputc
 .text.avr-libc
                0x00002d24       0xbc c:/program files (x86)/atmel/studio/7.0/toolchain/avr8/avr8-gnu-toolchain/bin/../lib/gcc/avr/5.4.0/../../../../avr/lib/avrxmega6\libc.a(ultoa_invert.o)
                0x00002d24                __ultoa_invert
                0x00002de0                . = ALIGN (0x2)
 *(.fini9)
 .fini9         0x00002de0        0x0 c:/program files (x86)/atmel/studio/7.0/toolchain/avr8/avr8-gnu-toolchain/bin/../lib/gcc/avr/5.4.0/avrxmega6\libgcc.a(_exit.o)
                0x00002de0                _exit
                0x00002de0                exit
 *(.fini9)
 *(.fini8)
 *(.fini8)
 *(.fini7)
 *(.fini7)
 *(.fini6)
 *(.fini6)
 *(.fini5)
 *(.fini5)
 *(.fini4)
 *(.fini4)
 *(.fini3)
 *(.fini3)
 *(.fini2)
 *(.fini2)
 *(.fini1)
 *(.fini1)
 *(.fini0)
 .fini0         0x00002de0        0x4 c:/program files (x86)/atmel/studio/7.0/toolchain/avr8/avr8-gnu-toolchain/bin/../lib/gcc/avr/5.4.0/avrxmega6\libgcc.a(_exit.o)
 *(.fini0)
                0x00002de4                _etext = .

.data           0x00802000       0x66 load address 0x00002de4
                0x00802000                PROVIDE (__data_start, .)
 *(.data)
 *(.data*)
 .data.sysfont  0x00802000        0x7 src/ASF/common/services/gfx_mono/sysfont.o
                0x00802000                sysfont
 .data.Ro       0x00802007        0x4 src/main.o
                0x00802007                Ro
 .data.SmokeCurve
                0x0080200b        0xc src/main.o
                0x0080200b                SmokeCurve
 .data.LPGCurve
                0x00802017        0xc src/main.o
                0x00802017                LPGCurve
 *(.gnu.linkonce.d*)
 *(.rodata)
 *(.rodata*)
 .rodata.str1.1
                0x00802023       0x42 src/main.o
 *(.gnu.linkonce.r*)
                0x00802066                . = ALIGN (0x2)
 *fill*         0x00802065        0x1 
                0x00802066                _edata = .
                0x00802066                PROVIDE (__data_end, .)

.bss            0x00802066      0x296
                0x00802066                PROVIDE (__bss_start, .)
 *(.bss)
 *(.bss*)
 .bss.ntc_sensor_samples.4861
                0x00802066        0x1 src/adc_sensors/adc_sensors.o
 .bss.light_sensor_samples.4860
                0x00802067        0x1 src/adc_sensors/adc_sensors.o
 .bss.light_sensor_sample
                0x00802068        0x2 src/adc_sensors/adc_sensors.o
                0x00802068                light_sensor_sample
 .bss.ntc_sensor_sample
                0x0080206a        0x2 src/adc_sensors/adc_sensors.o
                0x0080206a                ntc_sensor_sample
 .bss.light_sensor_data_ready
                0x0080206c        0x1 src/adc_sensors/adc_sensors.o
                0x0080206c                light_sensor_data_ready
 .bss.ntc_sensor_data_ready
                0x0080206d        0x1 src/adc_sensors/adc_sensors.o
                0x0080206d                ntc_sensor_data_ready
 .bss.framebuffer
                0x0080206e      0x200 src/ASF/common/services/gfx_mono/gfx_mono_c12832_a1z.o
 .bss.adcb_enable_count
                0x0080226e        0x1 src/ASF/xmega/drivers/adc/adc.o
 .bss.adca_enable_count
                0x0080226f        0x1 src/ASF/xmega/drivers/adc/adc.o
 .bss.fbpointer
                0x00802270        0x2 src/ASF/common/services/gfx_mono/gfx_mono_framebuffer.o
 .bss.strbuf    0x00802272       0x80 src/main.o
 *(COMMON)
 COMMON         0x008022f2        0x4 src/ASF/xmega/drivers/adc/adc.o
                0x008022f2                adcb_callback
                0x008022f4                adca_callback
 COMMON         0x008022f6        0x6 src/ASF/common/services/sleepmgr/xmega/sleepmgr.o
                0x008022f6                sleepmgr_locks
                0x008022fc                PROVIDE (__bss_end, .)
                0x00002de4                __data_load_start = LOADADDR (.data)
                0x00002e4a                __data_load_end = (__data_load_start + SIZEOF (.data))

.noinit         0x008022fc        0x0
                [!provide]                PROVIDE (__noinit_start, .)
 *(.noinit*)
                [!provide]                PROVIDE (__noinit_end, .)
                0x008022fc                _end = .
                [!provide]                PROVIDE (__heap_start, .)

.eeprom         0x00810000        0x0
 *(.eeprom*)
                0x00810000                __eeprom_end = .

.fuse
 *(.fuse)
 *(.lfuse)
 *(.hfuse)
 *(.efuse)

.lock
 *(.lock*)

.signature
 *(.signature*)

.user_signatures
 *(.user_signatures*)

.stab
 *(.stab)

.stabstr
 *(.stabstr)

.stab.excl
 *(.stab.excl)

.stab.exclstr
 *(.stab.exclstr)

.stab.index
 *(.stab.index)

.stab.indexstr
 *(.stab.indexstr)

.comment        0x00000000       0x5c
 *(.comment)
 .comment       0x00000000       0x30 src/adc_sensors/adc_sensors.o
                                 0x31 (size before relaxing)
 .comment       0x00000030       0x31 src/ASF/common/components/display/st7565r/st7565r.o
 .comment       0x00000030       0x31 src/ASF/common/services/gfx_mono/gfx_mono_c12832_a1z.o
 .comment       0x00000030       0x31 src/ASF/xmega/drivers/adc/adc.o
 .comment       0x00000030       0x31 src/ASF/xmega/drivers/usart/usart.o
 .comment       0x00000030       0x31 src/ASF/xmega/drivers/adc/xmega_aau/adc_aau.o
 .comment       0x00000030       0x31 src/ASF/common/services/spi/xmega_usart_spi/usart_spi.o
 .comment       0x00000030       0x31 src/ASF/common/services/sleepmgr/xmega/sleepmgr.o
 .comment       0x00000030       0x31 src/ASF/common/services/gfx_mono/gfx_mono_framebuffer.o
 .comment       0x00000030       0x31 src/ASF/common/services/gfx_mono/gfx_mono_generic.o
 .comment       0x00000030       0x31 src/ASF/common/services/clock/xmega/sysclk.o
 .comment       0x00000030       0x31 src/ASF/common/services/gfx_mono/gfx_mono_text.o
 .comment       0x00000030       0x31 src/ASF/common/services/gfx_mono/sysfont.o
 .comment       0x00000030       0x31 src/ASF/common/services/ioport/xmega/ioport_compat.o
 .comment       0x00000030       0x31 src/ASF/xmega/boards/xmega_a3bu_xplained/init.o
 .comment       0x00000030       0x31 src/main.o
 .comment       0x00000030       0x31 c:/program files (x86)/atmel/studio/7.0/toolchain/avr8/avr8-gnu-toolchain/bin/../lib/gcc/avr/5.4.0/../../../../avr/lib/avrxmega6\libc.a(snprintf.o)
 .comment       0x00000030       0x2c c:/program files (x86)/atmel/studio/7.0/toolchain/avr8/avr8-gnu-toolchain/bin/../lib/gcc/avr/5.4.0/../../../../avr/lib/avrxmega6\libc.a(vfprintf_std.o)
                                 0x2d (size before relaxing)
 .comment       0x0000005c       0x31 c:/program files (x86)/atmel/studio/7.0/toolchain/avr8/avr8-gnu-toolchain/bin/../lib/gcc/avr/5.4.0/../../../../avr/lib/avrxmega6\libc.a(fputc.o)

.note.gnu.avr.deviceinfo
                0x00000000       0x44
 .note.gnu.avr.deviceinfo
                0x00000000       0x44 C:/Program Files (x86)/Atmel/Studio/7.0/Packs/atmel/XMEGAA_DFP/1.3.146/gcc/dev/atxmega256a3bu/avrxmega6/crtatxmega256a3bu.o

.note.gnu.build-id
 *(.note.gnu.build-id)

.debug
 *(.debug)

.line
 *(.line)

.debug_srcinfo
 *(.debug_srcinfo)

.debug_sfnames
 *(.debug_sfnames)

.debug_aranges  0x00000000      0x460
 *(.debug_aranges)
 .debug_aranges
                0x00000000       0x50 src/adc_sensors/adc_sensors.o
 .debug_aranges
                0x00000050       0x28 src/ASF/common/components/display/st7565r/st7565r.o
 .debug_aranges
                0x00000078       0x60 src/ASF/common/services/gfx_mono/gfx_mono_c12832_a1z.o
 .debug_aranges
                0x000000d8       0x48 src/ASF/xmega/drivers/adc/adc.o
 .debug_aranges
                0x00000120       0x58 src/ASF/xmega/drivers/usart/usart.o
 .debug_aranges
                0x00000178       0x78 src/ASF/xmega/drivers/adc/xmega_aau/adc_aau.o
 .debug_aranges
                0x000001f0       0x48 src/ASF/common/services/spi/xmega_usart_spi/usart_spi.o
 .debug_aranges
                0x00000238       0x18 src/ASF/common/services/sleepmgr/xmega/sleepmgr.o
 .debug_aranges
                0x00000250       0x58 src/ASF/common/services/gfx_mono/gfx_mono_framebuffer.o
 .debug_aranges
                0x000002a8       0x58 src/ASF/common/services/gfx_mono/gfx_mono_generic.o
 .debug_aranges
                0x00000300       0x40 src/ASF/common/services/clock/xmega/sysclk.o
 .debug_aranges
                0x00000340       0x28 src/ASF/xmega/drivers/nvm/nvm_asm.o
 .debug_aranges
                0x00000368       0x40 src/ASF/common/services/gfx_mono/gfx_mono_text.o
 .debug_aranges
                0x000003a8       0x18 src/ASF/common/services/gfx_mono/sysfont.o
 .debug_aranges
                0x000003c0       0x20 src/ASF/common/services/ioport/xmega/ioport_compat.o
 .debug_aranges
                0x000003e0       0x20 src/ASF/xmega/boards/xmega_a3bu_xplained/init.o
 .debug_aranges
                0x00000400       0x60 src/main.o

.debug_pubnames
 *(.debug_pubnames)

.debug_info     0x00000000    0x112e6
 *(.debug_info .gnu.linkonce.wi.*)
 .debug_info    0x00000000     0x3379 C:/Program Files (x86)/Atmel/Studio/7.0/Packs/atmel/XMEGAA_DFP/1.3.146/gcc/dev/atxmega256a3bu/avrxmega6/crtatxmega256a3bu.o
 .debug_info    0x00003379     0x1214 src/adc_sensors/adc_sensors.o
 .debug_info    0x0000458d     0x1964 src/ASF/common/components/display/st7565r/st7565r.o
 .debug_info    0x00005ef1     0x1e01 src/ASF/common/services/gfx_mono/gfx_mono_c12832_a1z.o
 .debug_info    0x00007cf2      0xa6a src/ASF/xmega/drivers/adc/adc.o
 .debug_info    0x0000875c     0x2933 src/ASF/xmega/drivers/usart/usart.o
 .debug_info    0x0000b08f      0xe75 src/ASF/xmega/drivers/adc/xmega_aau/adc_aau.o
 .debug_info    0x0000bf04      0xb9d src/ASF/common/services/spi/xmega_usart_spi/usart_spi.o
 .debug_info    0x0000caa1      0x129 src/ASF/common/services/sleepmgr/xmega/sleepmgr.o
 .debug_info    0x0000cbca      0x487 src/ASF/common/services/gfx_mono/gfx_mono_framebuffer.o
 .debug_info    0x0000d051      0xc0a src/ASF/common/services/gfx_mono/gfx_mono_generic.o
 .debug_info    0x0000dc5b      0x71c src/ASF/common/services/clock/xmega/sysclk.o
 .debug_info    0x0000e377       0x85 src/ASF/xmega/drivers/nvm/nvm_asm.o
 .debug_info    0x0000e3fc      0x715 src/ASF/common/services/gfx_mono/gfx_mono_text.o
 .debug_info    0x0000eb11      0x1af src/ASF/common/services/gfx_mono/sysfont.o
 .debug_info    0x0000ecc0      0x121 src/ASF/common/services/ioport/xmega/ioport_compat.o
 .debug_info    0x0000ede1      0xb05 src/ASF/xmega/boards/xmega_a3bu_xplained/init.o
 .debug_info    0x0000f8e6     0x1a00 src/main.o

.debug_abbrev   0x00000000     0x56c6
 *(.debug_abbrev)
 .debug_abbrev  0x00000000     0x30c4 C:/Program Files (x86)/Atmel/Studio/7.0/Packs/atmel/XMEGAA_DFP/1.3.146/gcc/dev/atxmega256a3bu/avrxmega6/crtatxmega256a3bu.o
 .debug_abbrev  0x000030c4      0x397 src/adc_sensors/adc_sensors.o
 .debug_abbrev  0x0000345b      0x2a0 src/ASF/common/components/display/st7565r/st7565r.o
 .debug_abbrev  0x000036fb      0x385 src/ASF/common/services/gfx_mono/gfx_mono_c12832_a1z.o
 .debug_abbrev  0x00003a80      0x2bd src/ASF/xmega/drivers/adc/adc.o
 .debug_abbrev  0x00003d3d      0x3f5 src/ASF/xmega/drivers/usart/usart.o
 .debug_abbrev  0x00004132      0x329 src/ASF/xmega/drivers/adc/xmega_aau/adc_aau.o
 .debug_abbrev  0x0000445b      0x2d8 src/ASF/common/services/spi/xmega_usart_spi/usart_spi.o
 .debug_abbrev  0x00004733       0x84 src/ASF/common/services/sleepmgr/xmega/sleepmgr.o
 .debug_abbrev  0x000047b7      0x174 src/ASF/common/services/gfx_mono/gfx_mono_framebuffer.o
 .debug_abbrev  0x0000492b      0x1ac src/ASF/common/services/gfx_mono/gfx_mono_generic.o
 .debug_abbrev  0x00004ad7      0x218 src/ASF/common/services/clock/xmega/sysclk.o
 .debug_abbrev  0x00004cef       0x12 src/ASF/xmega/drivers/nvm/nvm_asm.o
 .debug_abbrev  0x00004d01      0x22b src/ASF/common/services/gfx_mono/gfx_mono_text.o
 .debug_abbrev  0x00004f2c       0xe2 src/ASF/common/services/gfx_mono/sysfont.o
 .debug_abbrev  0x0000500e       0x95 src/ASF/common/services/ioport/xmega/ioport_compat.o
 .debug_abbrev  0x000050a3      0x15c src/ASF/xmega/boards/xmega_a3bu_xplained/init.o
 .debug_abbrev  0x000051ff      0x4c7 src/main.o

.debug_line     0x00000000     0x9334
 *(.debug_line .debug_line.* .debug_line_end)
 .debug_line    0x00000000      0x39d C:/Program Files (x86)/Atmel/Studio/7.0/Packs/atmel/XMEGAA_DFP/1.3.146/gcc/dev/atxmega256a3bu/avrxmega6/crtatxmega256a3bu.o
 .debug_line    0x0000039d      0x886 src/adc_sensors/adc_sensors.o
 .debug_line    0x00000c23      0xac4 src/ASF/common/components/display/st7565r/st7565r.o
 .debug_line    0x000016e7      0xda8 src/ASF/common/services/gfx_mono/gfx_mono_c12832_a1z.o
 .debug_line    0x0000248f      0x7c6 src/ASF/xmega/drivers/adc/adc.o
 .debug_line    0x00002c55      0xc9e src/ASF/xmega/drivers/usart/usart.o
 .debug_line    0x000038f3      0x976 src/ASF/xmega/drivers/adc/xmega_aau/adc_aau.o
 .debug_line    0x00004269      0x7d7 src/ASF/common/services/spi/xmega_usart_spi/usart_spi.o
 .debug_line    0x00004a40      0x458 src/ASF/common/services/sleepmgr/xmega/sleepmgr.o
 .debug_line    0x00004e98      0x919 src/ASF/common/services/gfx_mono/gfx_mono_framebuffer.o
 .debug_line    0x000057b1      0xc05 src/ASF/common/services/gfx_mono/gfx_mono_generic.o
 .debug_line    0x000063b6      0x631 src/ASF/common/services/clock/xmega/sysclk.o
 .debug_line    0x000069e7      0x11f src/ASF/xmega/drivers/nvm/nvm_asm.o
 .debug_line    0x00006b06      0x9a3 src/ASF/common/services/gfx_mono/gfx_mono_text.o
 .debug_line    0x000074a9      0x7c3 src/ASF/common/services/gfx_mono/sysfont.o
 .debug_line    0x00007c6c      0x4b5 src/ASF/common/services/ioport/xmega/ioport_compat.o
 .debug_line    0x00008121      0x4e0 src/ASF/xmega/boards/xmega_a3bu_xplained/init.o
 .debug_line    0x00008601      0xd33 src/main.o

.debug_frame    0x00000000      0xfc0
 *(.debug_frame)
 .debug_frame   0x00000000       0xd8 src/adc_sensors/adc_sensors.o
 .debug_frame   0x000000d8       0x68 src/ASF/common/components/display/st7565r/st7565r.o
 .debug_frame   0x00000140      0x1b4 src/ASF/common/services/gfx_mono/gfx_mono_c12832_a1z.o
 .debug_frame   0x000002f4       0xbc src/ASF/xmega/drivers/adc/adc.o
 .debug_frame   0x000003b0      0x14c src/ASF/xmega/drivers/usart/usart.o
 .debug_frame   0x000004fc      0x3e4 src/ASF/xmega/drivers/adc/xmega_aau/adc_aau.o
 .debug_frame   0x000008e0       0x90 src/ASF/common/services/spi/xmega_usart_spi/usart_spi.o
 .debug_frame   0x00000970       0xd0 src/ASF/common/services/gfx_mono/gfx_mono_framebuffer.o
 .debug_frame   0x00000a40      0x214 src/ASF/common/services/gfx_mono/gfx_mono_generic.o
 .debug_frame   0x00000c54       0x94 src/ASF/common/services/clock/xmega/sysclk.o
 .debug_frame   0x00000ce8      0x100 src/ASF/common/services/gfx_mono/gfx_mono_text.o
 .debug_frame   0x00000de8       0x30 src/ASF/common/services/ioport/xmega/ioport_compat.o
 .debug_frame   0x00000e18       0x24 src/ASF/xmega/boards/xmega_a3bu_xplained/init.o
 .debug_frame   0x00000e3c      0x184 src/main.o

.debug_str      0x00000000    0x34712
 *(.debug_str)
 .debug_str     0x00000000     0x21e4 C:/Program Files (x86)/Atmel/Studio/7.0/Packs/atmel/XMEGAA_DFP/1.3.146/gcc/dev/atxmega256a3bu/avrxmega6/crtatxmega256a3bu.o
 .debug_str     0x000021e4    0x2ca5c src/adc_sensors/adc_sensors.o
                              0x2d2e2 (size before relaxing)
 .debug_str     0x0002ec40     0x14b1 src/ASF/common/components/display/st7565r/st7565r.o
                              0x2d09f (size before relaxing)
 .debug_str     0x000300f1      0xc05 src/ASF/common/services/gfx_mono/gfx_mono_c12832_a1z.o
                              0x2d9a0 (size before relaxing)
 .debug_str     0x00030cf6      0x1f4 src/ASF/xmega/drivers/adc/adc.o
                              0x2c80d (size before relaxing)
 .debug_str     0x00030eea      0x960 src/ASF/xmega/drivers/usart/usart.o
                              0x2cf96 (size before relaxing)
 .debug_str     0x0003184a      0x4fa src/ASF/xmega/drivers/adc/xmega_aau/adc_aau.o
                              0x2caa0 (size before relaxing)
 .debug_str     0x00031d44       0x87 src/ASF/common/services/spi/xmega_usart_spi/usart_spi.o
                              0x2c674 (size before relaxing)
 .debug_str     0x00031dcb       0x35 src/ASF/common/services/sleepmgr/xmega/sleepmgr.o
                              0x29862 (size before relaxing)
 .debug_str     0x00031e00       0xba src/ASF/common/services/gfx_mono/gfx_mono_framebuffer.o
                              0x2d5cf (size before relaxing)
 .debug_str     0x00031eba      0x213 src/ASF/common/services/gfx_mono/gfx_mono_generic.o
                              0x2d712 (size before relaxing)
 .debug_str     0x000320cd      0x232 src/ASF/common/services/clock/xmega/sysclk.o
                              0x2be92 (size before relaxing)
 .debug_str     0x000322ff      0x233 src/ASF/common/services/gfx_mono/gfx_mono_text.o
                              0x2d6a6 (size before relaxing)
 .debug_str     0x00032532     0x10b0 src/ASF/common/services/gfx_mono/sysfont.o
                              0x2e503 (size before relaxing)
 .debug_str     0x000335e2       0x77 src/ASF/common/services/ioport/xmega/ioport_compat.o
                              0x29b19 (size before relaxing)
 .debug_str     0x00033659       0xf7 src/ASF/xmega/boards/xmega_a3bu_xplained/init.o
                              0x2b7ba (size before relaxing)
 .debug_str     0x00033750      0xfc2 src/main.o
                              0x30ce2 (size before relaxing)

.debug_loc      0x00000000     0x73b9
 *(.debug_loc)
 .debug_loc     0x00000000      0x45f src/adc_sensors/adc_sensors.o
 .debug_loc     0x0000045f      0x7c9 src/ASF/common/components/display/st7565r/st7565r.o
 .debug_loc     0x00000c28     0x1382 src/ASF/common/services/gfx_mono/gfx_mono_c12832_a1z.o
 .debug_loc     0x00001faa      0x2b3 src/ASF/xmega/drivers/adc/adc.o
 .debug_loc     0x0000225d      0xe14 src/ASF/xmega/drivers/usart/usart.o
 .debug_loc     0x00003071      0xd3c src/ASF/xmega/drivers/adc/xmega_aau/adc_aau.o
 .debug_loc     0x00003dad      0x56c src/ASF/common/services/spi/xmega_usart_spi/usart_spi.o
 .debug_loc     0x00004319      0x61c src/ASF/common/services/gfx_mono/gfx_mono_framebuffer.o
 .debug_loc     0x00004935     0x11c5 src/ASF/common/services/gfx_mono/gfx_mono_generic.o
 .debug_loc     0x00005afa      0x2c5 src/ASF/common/services/clock/xmega/sysclk.o
 .debug_loc     0x00005dbf      0x9a2 src/ASF/common/services/gfx_mono/gfx_mono_text.o
 .debug_loc     0x00006761       0x66 src/ASF/common/services/ioport/xmega/ioport_compat.o
 .debug_loc     0x000067c7      0x3fa src/ASF/xmega/boards/xmega_a3bu_xplained/init.o
 .debug_loc     0x00006bc1      0x7f8 src/main.o

.debug_macinfo
 *(.debug_macinfo)

.debug_weaknames
 *(.debug_weaknames)

.debug_funcnames
 *(.debug_funcnames)

.debug_typenames
 *(.debug_typenames)

.debug_varnames
 *(.debug_varnames)

.debug_pubtypes
 *(.debug_pubtypes)

.debug_ranges   0x00000000      0x530
 *(.debug_ranges)
 .debug_ranges  0x00000000       0x40 src/adc_sensors/adc_sensors.o
 .debug_ranges  0x00000040       0x18 src/ASF/common/components/display/st7565r/st7565r.o
 .debug_ranges  0x00000058      0x188 src/ASF/common/services/gfx_mono/gfx_mono_c12832_a1z.o
 .debug_ranges  0x000001e0       0x38 src/ASF/xmega/drivers/adc/adc.o
 .debug_ranges  0x00000218       0x80 src/ASF/xmega/drivers/usart/usart.o
 .debug_ranges  0x00000298       0x68 src/ASF/xmega/drivers/adc/xmega_aau/adc_aau.o
 .debug_ranges  0x00000300       0x98 src/ASF/common/services/spi/xmega_usart_spi/usart_spi.o
 .debug_ranges  0x00000398       0x48 src/ASF/common/services/gfx_mono/gfx_mono_framebuffer.o
 .debug_ranges  0x000003e0       0x48 src/ASF/common/services/gfx_mono/gfx_mono_generic.o
 .debug_ranges  0x00000428       0x30 src/ASF/common/services/clock/xmega/sysclk.o
 .debug_ranges  0x00000458       0x20 src/ASF/xmega/drivers/nvm/nvm_asm.o
 .debug_ranges  0x00000478       0x30 src/ASF/common/services/gfx_mono/gfx_mono_text.o
 .debug_ranges  0x000004a8       0x10 src/ASF/common/services/ioport/xmega/ioport_compat.o
 .debug_ranges  0x000004b8       0x10 src/ASF/xmega/boards/xmega_a3bu_xplained/init.o
 .debug_ranges  0x000004c8       0x68 src/main.o

.debug_macro    0x00000000     0xca44
 *(.debug_macro)
 .debug_macro   0x00000000      0x245 src/adc_sensors/adc_sensors.o
 .debug_macro   0x00000245      0xa9c src/adc_sensors/adc_sensors.o
 .debug_macro   0x00000ce1       0x10 src/adc_sensors/adc_sensors.o
 .debug_macro   0x00000cf1      0x1c9 src/adc_sensors/adc_sensors.o
 .debug_macro   0x00000eba      0x2fc src/adc_sensors/adc_sensors.o
 .debug_macro   0x000011b6       0x9e src/adc_sensors/adc_sensors.o
 .debug_macro   0x00001254     0x62b7 src/adc_sensors/adc_sensors.o
 .debug_macro   0x0000750b       0x9a src/adc_sensors/adc_sensors.o
 .debug_macro   0x000075a5       0xf1 src/adc_sensors/adc_sensors.o
 .debug_macro   0x00007696       0x34 src/adc_sensors/adc_sensors.o
 .debug_macro   0x000076ca       0x16 src/adc_sensors/adc_sensors.o
 .debug_macro   0x000076e0       0x18 src/adc_sensors/adc_sensors.o
 .debug_macro   0x000076f8       0x5e src/adc_sensors/adc_sensors.o
 .debug_macro   0x00007756       0x10 src/adc_sensors/adc_sensors.o
 .debug_macro   0x00007766       0x22 src/adc_sensors/adc_sensors.o
 .debug_macro   0x00007788      0x16d src/adc_sensors/adc_sensors.o
 .debug_macro   0x000078f5       0x1c src/adc_sensors/adc_sensors.o
 .debug_macro   0x00007911       0x35 src/adc_sensors/adc_sensors.o
 .debug_macro   0x00007946       0x66 src/adc_sensors/adc_sensors.o
 .debug_macro   0x000079ac      0x71d src/adc_sensors/adc_sensors.o
 .debug_macro   0x000080c9       0x96 src/adc_sensors/adc_sensors.o
 .debug_macro   0x0000815f       0x17 src/adc_sensors/adc_sensors.o
 .debug_macro   0x00008176      0x250 src/adc_sensors/adc_sensors.o
 .debug_macro   0x000083c6       0x76 src/adc_sensors/adc_sensors.o
 .debug_macro   0x0000843c       0x16 src/adc_sensors/adc_sensors.o
 .debug_macro   0x00008452      0x6d9 src/adc_sensors/adc_sensors.o
 .debug_macro   0x00008b2b       0x10 src/adc_sensors/adc_sensors.o
 .debug_macro   0x00008b3b      0x175 src/adc_sensors/adc_sensors.o
 .debug_macro   0x00008cb0       0x40 src/adc_sensors/adc_sensors.o
 .debug_macro   0x00008cf0       0x69 src/adc_sensors/adc_sensors.o
 .debug_macro   0x00008d59       0x31 src/adc_sensors/adc_sensors.o
 .debug_macro   0x00008d8a       0xe4 src/adc_sensors/adc_sensors.o
 .debug_macro   0x00008e6e       0x10 src/adc_sensors/adc_sensors.o
 .debug_macro   0x00008e7e       0x20 src/adc_sensors/adc_sensors.o
 .debug_macro   0x00008e9e       0x10 src/adc_sensors/adc_sensors.o
 .debug_macro   0x00008eae       0x42 src/adc_sensors/adc_sensors.o
 .debug_macro   0x00008ef0       0x22 src/adc_sensors/adc_sensors.o
 .debug_macro   0x00008f12      0x2df src/adc_sensors/adc_sensors.o
 .debug_macro   0x000091f1      0x2ff src/adc_sensors/adc_sensors.o
 .debug_macro   0x000094f0       0x79 src/adc_sensors/adc_sensors.o
 .debug_macro   0x00009569       0x2f src/adc_sensors/adc_sensors.o
 .debug_macro   0x00009598      0x154 src/adc_sensors/adc_sensors.o
 .debug_macro   0x000096ec       0xe3 src/adc_sensors/adc_sensors.o
 .debug_macro   0x000097cf      0x276 src/ASF/common/components/display/st7565r/st7565r.o
 .debug_macro   0x00009a45       0x82 src/ASF/common/components/display/st7565r/st7565r.o
 .debug_macro   0x00009ac7      0x102 src/ASF/common/components/display/st7565r/st7565r.o
 .debug_macro   0x00009bc9       0x28 src/ASF/common/components/display/st7565r/st7565r.o
 .debug_macro   0x00009bf1       0x22 src/ASF/common/components/display/st7565r/st7565r.o
 .debug_macro   0x00009c13       0x3a src/ASF/common/components/display/st7565r/st7565r.o
 .debug_macro   0x00009c4d       0xf6 src/ASF/common/components/display/st7565r/st7565r.o
 .debug_macro   0x00009d43       0x34 src/ASF/common/components/display/st7565r/st7565r.o
 .debug_macro   0x00009d77       0x2e src/ASF/common/components/display/st7565r/st7565r.o
 .debug_macro   0x00009da5      0x2ba src/ASF/common/services/gfx_mono/gfx_mono_c12832_a1z.o
 .debug_macro   0x0000a05f       0x75 src/ASF/common/services/gfx_mono/gfx_mono_c12832_a1z.o
 .debug_macro   0x0000a0d4       0x88 src/ASF/common/services/gfx_mono/gfx_mono_c12832_a1z.o
 .debug_macro   0x0000a15c      0x22f src/ASF/xmega/drivers/adc/adc.o
 .debug_macro   0x0000a38b      0x221 src/ASF/xmega/drivers/usart/usart.o
 .debug_macro   0x0000a5ac      0x302 src/ASF/xmega/drivers/usart/usart.o
 .debug_macro   0x0000a8ae      0x22f src/ASF/xmega/drivers/adc/xmega_aau/adc_aau.o
 .debug_macro   0x0000aadd      0x234 src/ASF/common/services/spi/xmega_usart_spi/usart_spi.o
 .debug_macro   0x0000ad11      0x1a3 src/ASF/common/services/sleepmgr/xmega/sleepmgr.o
 .debug_macro   0x0000aeb4      0x2ae src/ASF/common/services/gfx_mono/gfx_mono_framebuffer.o
 .debug_macro   0x0000b162      0x2ae src/ASF/common/services/gfx_mono/gfx_mono_generic.o
 .debug_macro   0x0000b410      0x1db src/ASF/common/services/clock/xmega/sysclk.o
 .debug_macro   0x0000b5eb       0x26 src/ASF/common/services/clock/xmega/sysclk.o
 .debug_macro   0x0000b611      0x2d5 src/ASF/common/services/gfx_mono/gfx_mono_text.o
 .debug_macro   0x0000b8e6       0xaa src/ASF/common/services/gfx_mono/gfx_mono_text.o
 .debug_macro   0x0000b990      0x2db src/ASF/common/services/gfx_mono/sysfont.o
 .debug_macro   0x0000bc6b       0x3a src/ASF/common/services/gfx_mono/sysfont.o
 .debug_macro   0x0000bca5      0x193 src/ASF/common/services/ioport/xmega/ioport_compat.o
 .debug_macro   0x0000be38      0x1b5 src/ASF/xmega/boards/xmega_a3bu_xplained/init.o
 .debug_macro   0x0000bfed       0x2e src/ASF/xmega/boards/xmega_a3bu_xplained/init.o
 .debug_macro   0x0000c01b      0x2d9 src/ASF/xmega/boards/xmega_a3bu_xplained/init.o
 .debug_macro   0x0000c2f4      0x3ea src/main.o
 .debug_macro   0x0000c6de       0x34 src/main.o
 .debug_macro   0x0000c712       0x16 src/main.o
 .debug_macro   0x0000c728       0x46 src/main.o
 .debug_macro   0x0000c76e       0x1c src/main.o
 .debug_macro   0x0000c78a       0x58 src/main.o
 .debug_macro   0x0000c7e2       0x10 src/main.o
 .debug_macro   0x0000c7f2       0xf2 src/main.o
 .debug_macro   0x0000c8e4      0x160 src/main.o
OUTPUT(UTS2.elf elf32-avr)
LOAD linker stubs

.BOOT           0x00040000        0x0
